BL51 BANKED LINKER/LOCATER V6.22                                                        05/19/2022  10:01:03  PAGE 1


BL51 BANKED LINKER/LOCATER V6.22, INVOKED BY:
C:\KEIL_V5\C51\BIN\BL51.EXE .\Objects\main.obj, .\Objects\i2c.obj, .\Objects\OPTIONS_SN8F5835.obj TO .\Objects\SN8F5835_
>> Test Code PRINT (.\Listings\SN8F5835_Test Code.m51) RAMSIZE (256)


MEMORY MODEL: SMALL


INPUT MODULES INCLUDED:
  .\Objects\main.obj (MAIN)
  .\Objects\i2c.obj (I2C)
  .\Objects\OPTIONS_SN8F5835.obj (OPTIONS_SN8F5835)
  C:\KEIL_V5\C51\LIB\C51S.LIB (?C_STARTUP)
  C:\KEIL_V5\C51\LIB\C51S.LIB (?C?CLDPTR)
  C:\KEIL_V5\C51\LIB\C51S.LIB (?C?CSTPTR)
  C:\KEIL_V5\C51\LIB\C51S.LIB (?C?CCASE)
  C:\KEIL_V5\C51\LIB\C51S.LIB (?C_INIT)


LINK MAP OF MODULE:  .\Objects\SN8F5835_Test Code (MAIN)


            TYPE    BASE      LENGTH    RELOCATION   SEGMENT NAME
            -----------------------------------------------------

            * * * * * * *   D A T A   M E M O R Y   * * * * * * *
            REG     0000H     0008H     ABSOLUTE     "REG BANK 0"
            DATA    0008H     0016H     UNIT         ?DT?I2C
                    001EH     0002H                  *** GAP ***
            BIT     0020H.0   0000H.1   UNIT         _BIT_GROUP_
                    0020H.1   0000H.7                *** GAP ***
            DATA    0021H     001EH     UNIT         ?DT?MAIN
            DATA    003FH     0005H     UNIT         _DATA_GROUP_
            IDATA   0044H     0001H     UNIT         ?STACK

            * * * * * * *  X D A T A   M E M O R Y  * * * * * * *
                    0000H     F000H                  *** GAP ***
            XDATA   F000H     0001H     ABSOLUTE     
            XDATA   F001H     0001H     ABSOLUTE     
            XDATA   F002H     0001H     ABSOLUTE     
            XDATA   F003H     0001H     ABSOLUTE     
            XDATA   F004H     0001H     ABSOLUTE     
            XDATA   F005H     0001H     ABSOLUTE     
            XDATA   F006H     0001H     ABSOLUTE     
            XDATA   F007H     0001H     ABSOLUTE     
            XDATA   F008H     0001H     ABSOLUTE     
            XDATA   F009H     0001H     ABSOLUTE     
            XDATA   F00AH     0001H     ABSOLUTE     
            XDATA   F00BH     0001H     ABSOLUTE     
            XDATA   F00CH     0001H     ABSOLUTE     
            XDATA   F00DH     0001H     ABSOLUTE     
            XDATA   F00EH     0001H     ABSOLUTE     
            XDATA   F00FH     0001H     ABSOLUTE     
            XDATA   F010H     0001H     ABSOLUTE     
            XDATA   F011H     0001H     ABSOLUTE     
            XDATA   F012H     0001H     ABSOLUTE     
            XDATA   F013H     0001H     ABSOLUTE     
            XDATA   F014H     0001H     ABSOLUTE     
BL51 BANKED LINKER/LOCATER V6.22                                                      05/19/2022  10:01:03  PAGE 2


                    F015H     0001H                  *** GAP ***
            XDATA   F016H     0001H     ABSOLUTE     
            XDATA   F017H     0001H     ABSOLUTE     
            XDATA   F018H     0001H     ABSOLUTE     
            XDATA   F019H     0001H     ABSOLUTE     
            XDATA   F01AH     0001H     ABSOLUTE     
            XDATA   F01BH     0001H     ABSOLUTE     
            XDATA   F01CH     0001H     ABSOLUTE     
            XDATA   F01DH     0001H     ABSOLUTE     
            XDATA   F01EH     0001H     ABSOLUTE     
            XDATA   F01FH     0001H     ABSOLUTE     
            XDATA   F020H     0001H     ABSOLUTE     
            XDATA   F021H     0001H     ABSOLUTE     
            XDATA   F022H     0001H     ABSOLUTE     
            XDATA   F023H     0001H     ABSOLUTE     
            XDATA   F024H     0001H     ABSOLUTE     
            XDATA   F025H     0001H     ABSOLUTE     
            XDATA   F026H     0001H     ABSOLUTE     
            XDATA   F027H     0001H     ABSOLUTE     
            XDATA   F028H     0001H     ABSOLUTE     
            XDATA   F029H     0001H     ABSOLUTE     
                    F02AH     0001H                  *** GAP ***
            XDATA   F02BH     0001H     ABSOLUTE     
            XDATA   F02CH     0001H     ABSOLUTE     
            XDATA   F02DH     0001H     ABSOLUTE     
            XDATA   F02EH     0001H     ABSOLUTE     
            XDATA   F02FH     0001H     ABSOLUTE     
            XDATA   F030H     0001H     ABSOLUTE     
            XDATA   F031H     0001H     ABSOLUTE     
            XDATA   F032H     0001H     ABSOLUTE     
            XDATA   F033H     0001H     ABSOLUTE     

            * * * * * * *   C O D E   M E M O R Y   * * * * * * *
            CODE    0000H     0003H     ABSOLUTE     
            CODE    0003H     0037H     UNIT         ?PR?I2C_INITMASTERTX?I2C
                    003AH     0009H                  *** GAP ***
            CODE    0043H     0003H     ABSOLUTE     
            CODE    0046H     021CH     UNIT         ?PR?I2C_EXECUTETRANSMISSION?I2C
            CODE    0262H     008CH     UNIT         ?C_C51STARTUP
            CODE    02EEH     005FH     UNIT         ?PR?MAIN?MAIN
            CODE    034DH     0051H     UNIT         ?C?LIB_CODE
            CODE    039EH     0037H     UNIT         ?PR?I2C_INITMASTERRX?I2C
            CODE    03D5H     002BH     UNIT         ?PR?ISR_I2C?I2C
            CODE    0400H     0025H     UNIT         ?PR?_I2C_CONFIGUREREGISTER?I2C
            CODE    0425H     0020H     UNIT         ?PR?I2C_REPEATMASTER?I2C
            CODE    0445H     0019H     UNIT         ?PR?GPIO_INITIALIZATION?I2C
            CODE    045EH     0012H     UNIT         ?PR?I2C_CHECKTRANSDATASTOP?I2C
            CODE    0470H     0012H     UNIT         ?PR?I2C_CHECKRECIDATASTOP?I2C
            CODE    0482H     0010H     UNIT         ?PR?I2C_CHECKTRANSDATADONE?I2C
            CODE    0492H     0010H     UNIT         ?PR?I2C_CHECKRECIDATADONE?I2C
            CODE    04A2H     000DH     UNIT         ?C_INITSEG
                    04AFH     7B41H                  *** GAP ***
            CODE    7FF0H     0002H     ABSOLUTE     
                    7FF2H     0004H                  *** GAP ***
            CODE    7FF6H     000AH     ABSOLUTE     


BL51 BANKED LINKER/LOCATER V6.22                                                      05/19/2022  10:01:03  PAGE 3



OVERLAY MAP OF MODULE:   .\Objects\SN8F5835_Test Code (MAIN)


SEGMENT                                    BIT_GROUP          DATA_GROUP 
  +--> CALLED SEGMENT                   START    LENGTH     START    LENGTH
---------------------------------------------------------------------------
?PR?ISR_I2C?I2C                         -----    -----      -----    -----
  +--> ?PR?I2C_EXECUTETRANSMISSION?I2C

*** NEW ROOT ***************************************************

?C_C51STARTUP                           -----    -----      -----    -----
  +--> ?PR?MAIN?MAIN
  +--> ?C_INITSEG

?PR?MAIN?MAIN                           -----    -----      -----    -----
  +--> ?PR?GPIO_INITIALIZATION?I2C
  +--> ?PR?_I2C_CONFIGUREREGISTER?I2C
  +--> ?PR?I2C_INITMASTERTX?I2C
  +--> ?PR?I2C_INITMASTERRX?I2C
  +--> ?PR?I2C_CHECKTRANSDATADONE?I2C
  +--> ?PR?I2C_CHECKTRANSDATASTOP?I2C
  +--> ?PR?I2C_REPEATMASTER?I2C
  +--> ?PR?I2C_CHECKRECIDATADONE?I2C
  +--> ?PR?I2C_CHECKRECIDATASTOP?I2C

?PR?_I2C_CONFIGUREREGISTER?I2C          -----    -----      003FH    0004H

?PR?I2C_INITMASTERTX?I2C                0020H.0  0000H.1    003FH    0005H

?PR?I2C_INITMASTERRX?I2C                0020H.0  0000H.1    003FH    0005H

?PR?I2C_CHECKTRANSDATADONE?I2C          0020H.0  0000H.1    -----    -----

?PR?I2C_CHECKTRANSDATASTOP?I2C          0020H.0  0000H.1    -----    -----

?PR?I2C_CHECKRECIDATADONE?I2C           0020H.0  0000H.1    -----    -----

?PR?I2C_CHECKRECIDATASTOP?I2C           0020H.0  0000H.1    -----    -----



SYMBOL TABLE OF MODULE:  .\Objects\SN8F5835_Test Code (MAIN)

  VALUE           TYPE          NAME
  ----------------------------------

  -------         MODULE        MAIN
  C:0000H         SYMBOL        _ICE_DUMMY_
  X:F003H         PUBLIC        PW1YL
  X:F017H         PUBLIC        PW2YL
  D:0080H         PUBLIC        P0
  X:F031H         PUBLIC        PW3YL
  D:0090H         PUBLIC        P1
  D:00B0H         PUBLIC        P3
  D:00C8H         PUBLIC        P4
BL51 BANKED LINKER/LOCATER V6.22                                                      05/19/2022  10:01:03  PAGE 4


  D:00A0H         PUBLIC        TTCON
  D:00A8H         PUBLIC        IEN0
  D:00B8H         PUBLIC        IEN1
  X:F004H         PUBLIC        PW10DH
  X:F018H         PUBLIC        PW20DH
  X:F006H         PUBLIC        PW11DH
  X:F01AH         PUBLIC        PW21DH
  X:F00CH         PUBLIC        PW30DH
  X:F008H         PUBLIC        PW12DH
  X:F01CH         PUBLIC        PW22DH
  X:F00EH         PUBLIC        PW31DH
  X:F00AH         PUBLIC        PW13DH
  X:F01EH         PUBLIC        PW23DH
  X:F010H         PUBLIC        PW32DH
  X:F005H         PUBLIC        PW10DL
  X:F019H         PUBLIC        PW20DL
  X:F012H         PUBLIC        PW33DH
  X:F007H         PUBLIC        PW11DL
  X:F01BH         PUBLIC        PW21DL
  X:F00DH         PUBLIC        PW30DL
  X:F009H         PUBLIC        PW12DL
  X:F01DH         PUBLIC        PW22DL
  X:F00FH         PUBLIC        PW31DL
  X:F00BH         PUBLIC        PW13DL
  X:F01FH         PUBLIC        PW23DL
  X:F011H         PUBLIC        PW32DL
  X:F013H         PUBLIC        PW33DL
  X:F000H         PUBLIC        PW1M
  C:02EEH         PUBLIC        main
  X:F014H         PUBLIC        PW2M
  X:F02DH         PUBLIC        HIDR
  X:F028H         PUBLIC        P0UR
  X:F001H         PUBLIC        PW3M
  X:F029H         PUBLIC        P1UR
  X:F02BH         PUBLIC        P3UR
  X:F02CH         PUBLIC        P4UR
  D:00D8H         PUBLIC        CSCON4
  D:0088H         PUBLIC        TCON
  X:F027H         PUBLIC        TSWA
  X:F026H         PUBLIC        TSWB
  X:F025H         PUBLIC        TSWD
  B:00A8H.7       PUBLIC        EAL
  X:F02EH         PUBLIC        CSADB1H
  X:F024H         PUBLIC        TSWY
  X:F032H         PUBLIC        CSADB2H
  X:F02FH         PUBLIC        CSADB1L
  X:F033H         PUBLIC        CSADB2L
  D:0098H         PUBLIC        S0CON
  D:0021H         PUBLIC        bI2C_RxDataBuf
  D:002BH         PUBLIC        bI2C_TxDataBuf
  X:F022H         PUBLIC        MINCS0H
  X:F020H         PUBLIC        MAXCS0H
  X:F023H         PUBLIC        MINCS0L
  D:0035H         PUBLIC        bMN_DataBuf
  X:F021H         PUBLIC        MAXCS0L
  X:F002H         PUBLIC        PW1YH
  D:00D0H         PUBLIC        PSW
BL51 BANKED LINKER/LOCATER V6.22                                                      05/19/2022  10:01:03  PAGE 5


  X:F016H         PUBLIC        PW2YH
  X:F030H         PUBLIC        PW3YH
  D:00C0H         PUBLIC        IRCON
  -------         PROC          MAIN
  C:02EEH         LINE#         38
  C:02EEH         LINE#         39
  C:02EEH         LINE#         41
  C:02F1H         LINE#         44
  C:02FDH         LINE#         47
  C:02FFH         LINE#         50
  C:0313H         LINE#         53
  C:0327H         LINE#         55
  C:0327H         LINE#         56
  C:0327H         LINE#         58
  C:032CH         LINE#         59
  C:032CH         LINE#         60
  C:032CH         LINE#         61
  C:032EH         LINE#         63
  C:032EH         LINE#         65
  C:0333H         LINE#         66
  C:0333H         LINE#         67
  C:0336H         LINE#         68
  C:0336H         LINE#         69
  C:0336H         LINE#         72
  C:033BH         LINE#         73
  C:033BH         LINE#         74
  C:033EH         LINE#         76
  C:0341H         LINE#         77
  C:0343H         LINE#         79
  C:0343H         LINE#         81
  C:0348H         LINE#         82
  C:0348H         LINE#         83
  C:034BH         LINE#         84
  C:034BH         LINE#         85
  C:034BH         LINE#         86
  -------         ENDPROC       MAIN
  -------         ENDMOD        MAIN

  -------         MODULE        I2C
  C:0000H         SYMBOL        _ICE_DUMMY_
  D:0080H         PUBLIC        P0
  D:0090H         PUBLIC        P1
  D:00B0H         PUBLIC        P3
  D:00C8H         PUBLIC        P4
  D:0008H         PUBLIC        stI2C_RxHardware
  D:0012H         PUBLIC        stI2C_TxHardware
  D:00A0H         PUBLIC        TTCON
  C:0046H         PUBLIC        I2C_ExecuteTransmission
  C:0492H         PUBLIC        I2C_CheckReciDataDone
  D:00A8H         PUBLIC        IEN0
  D:00B8H         PUBLIC        IEN1
  C:0482H         PUBLIC        I2C_CheckTransDataDone
  C:0400H         PUBLIC        _I2C_ConfigureRegister
  D:00DBH         PUBLIC        I2CADR
  D:00DAH         PUBLIC        I2CDAT
  D:00DCH         PUBLIC        I2CCON
  D:00DDH         PUBLIC        I2CSTA
BL51 BANKED LINKER/LOCATER V6.22                                                      05/19/2022  10:01:03  PAGE 6


  D:001CH         PUBLIC        stI2C_MasterHardware
  C:0470H         PUBLIC        I2C_CheckReciDataStop
  D:00D8H         PUBLIC        CSCON4
  C:03D5H         PUBLIC        ISR_I2c
  C:045EH         PUBLIC        I2C_CheckTransDataStop
  D:0088H         PUBLIC        TCON
  D:00DEH         PUBLIC        SMBSEL
  D:00F9H         PUBLIC        P0M
  D:00FAH         PUBLIC        P1M
  D:00FBH         PUBLIC        P3M
  C:039EH         PUBLIC        I2C_InitMasterRX
  D:00FCH         PUBLIC        P4M
  C:0003H         PUBLIC        I2C_InitMasterTX
  C:0445H         PUBLIC        GPIO_Initialization
  D:0098H         PUBLIC        S0CON
  C:0425H         PUBLIC        I2C_RepeatMaster
  D:00D0H         PUBLIC        PSW
  D:00C0H         PUBLIC        IRCON
  -------         PROC          GPIO_INITIALIZATION
  C:0445H         LINE#         41
  C:0445H         LINE#         42
  C:0445H         LINE#         44
  C:044BH         LINE#         45
  C:0451H         LINE#         46
  C:0457H         LINE#         47
  C:045DH         LINE#         48
  -------         ENDPROC       GPIO_INITIALIZATION
  -------         PROC          _I2C_CONFIGUREREGISTER
  D:0007H         SYMBOL        bMuxNum
  D:0005H         SYMBOL        bClockDiv
  D:0003H         SYMBOL        bSelfAddress
  D:0042H         SYMBOL        bMateAddress
  C:0400H         LINE#         56
  C:0400H         LINE#         57
  C:0400H         LINE#         59
  C:0403H         LINE#         62
  C:0406H         LINE#         63
  C:0406H         LINE#         64
  C:040CH         LINE#         65
  C:040EH         LINE#         67
  C:040EH         LINE#         68
  C:0414H         LINE#         69
  C:0414H         LINE#         70
  C:0419H         LINE#         73
  C:041EH         LINE#         74
  C:0421H         LINE#         77
  C:0424H         LINE#         78
  -------         ENDPROC       _I2C_CONFIGUREREGISTER
  -------         PROC          I2C_INITMASTERTX
  B:0020H.0       SYMBOL        fTxRxSel
  D:003FH         SYMBOL        bptrDataBuf
  D:0042H         SYMBOL        dbLength
  C:0003H         LINE#         86
  C:0003H         LINE#         87
  C:0003H         LINE#         88
  C:0006H         LINE#         89
  C:0006H         LINE#         90
BL51 BANKED LINKER/LOCATER V6.22                                                      05/19/2022  10:01:03  PAGE 7


  C:0012H         LINE#         91
  C:0027H         LINE#         92
  C:0030H         LINE#         93
  C:0033H         LINE#         94
  C:0033H         LINE#         96
  C:0036H         LINE#         97
  C:0039H         LINE#         98
  -------         ENDPROC       I2C_INITMASTERTX
  -------         PROC          I2C_INITMASTERRX
  B:0020H.0       SYMBOL        fTxRxSel
  D:003FH         SYMBOL        bptrDataBuf
  D:0042H         SYMBOL        dbLength
  C:039EH         LINE#         105
  C:039EH         LINE#         106
  C:039EH         LINE#         107
  C:03A1H         LINE#         108
  C:03A1H         LINE#         109
  C:03ADH         LINE#         110
  C:03C2H         LINE#         111
  C:03CBH         LINE#         112
  C:03CEH         LINE#         113
  C:03CEH         LINE#         115
  C:03D1H         LINE#         116
  C:03D4H         LINE#         117
  -------         ENDPROC       I2C_INITMASTERRX
  -------         PROC          I2C_REPEATMASTER
  C:0425H         LINE#         123
  C:0425H         LINE#         124
  C:0425H         LINE#         125
  C:042AH         LINE#         126
  C:042AH         LINE#         127
  C:0433H         LINE#         128
  C:0435H         LINE#         130
  C:0435H         LINE#         131
  C:043EH         LINE#         132
  C:043EH         LINE#         134
  C:0441H         LINE#         135
  C:0444H         LINE#         136
  -------         ENDPROC       I2C_REPEATMASTER
  -------         PROC          I2C_CHECKTRANSDATADONE
  -------         DO            
  B:0020H.0       SYMBOL        fDoneFlag
  -------         ENDDO         
  C:0482H         LINE#         143
  C:0482H         LINE#         144
  C:0482H         LINE#         145
  C:0484H         LINE#         146
  C:0489H         LINE#         147
  C:0489H         LINE#         148
  C:048CH         LINE#         149
  C:048FH         LINE#         150
  C:048FH         LINE#         151
  C:0491H         LINE#         152
  -------         ENDPROC       I2C_CHECKTRANSDATADONE
  -------         PROC          I2C_CHECKTRANSDATASTOP
  -------         DO            
  B:0020H.0       SYMBOL        fNACKFlag
BL51 BANKED LINKER/LOCATER V6.22                                                      05/19/2022  10:01:03  PAGE 8


  -------         ENDDO         
  C:045EH         LINE#         159
  C:045EH         LINE#         160
  C:045EH         LINE#         161
  C:0460H         LINE#         162
  C:0465H         LINE#         163
  C:0465H         LINE#         164
  C:046AH         LINE#         165
  C:046DH         LINE#         166
  C:046DH         LINE#         167
  C:046FH         LINE#         168
  -------         ENDPROC       I2C_CHECKTRANSDATASTOP
  -------         PROC          I2C_CHECKRECIDATADONE
  -------         DO            
  B:0020H.0       SYMBOL        fDoneFlag
  -------         ENDDO         
  C:0492H         LINE#         175
  C:0492H         LINE#         176
  C:0492H         LINE#         177
  C:0494H         LINE#         178
  C:0499H         LINE#         179
  C:0499H         LINE#         180
  C:049CH         LINE#         181
  C:049FH         LINE#         182
  C:049FH         LINE#         183
  C:04A1H         LINE#         184
  -------         ENDPROC       I2C_CHECKRECIDATADONE
  -------         PROC          I2C_CHECKRECIDATASTOP
  -------         DO            
  B:0020H.0       SYMBOL        fNACKFlag
  -------         ENDDO         
  C:0470H         LINE#         191
  C:0470H         LINE#         192
  C:0470H         LINE#         193
  C:0472H         LINE#         194
  C:0477H         LINE#         195
  C:0477H         LINE#         196
  C:047CH         LINE#         197
  C:047FH         LINE#         198
  C:047FH         LINE#         199
  C:0481H         LINE#         200
  -------         ENDPROC       I2C_CHECKRECIDATASTOP
  -------         PROC          I2C_EXECUTETRANSMISSION
  C:0046H         LINE#         207
  C:0046H         LINE#         208
  C:0046H         LINE#         209
  C:0089H         LINE#         210
  C:0089H         LINE#         213
  C:0089H         LINE#         214
  C:0089H         LINE#         215
  C:0089H         LINE#         216
  C:0089H         LINE#         217
  C:008CH         LINE#         219
  C:0098H         LINE#         220
  C:009BH         LINE#         226
  C:009BH         LINE#         227
  C:009EH         LINE#         228
BL51 BANKED LINKER/LOCATER V6.22                                                      05/19/2022  10:01:03  PAGE 9


  C:00B1H         LINE#         229
  C:00CCH         LINE#         230
  C:00CCH         LINE#         231
  C:00CCH         LINE#         232
  C:00CCH         LINE#         233
  C:00CCH         LINE#         234
  C:00CEH         LINE#         235
  C:00CEH         LINE#         236
  C:00D1H         LINE#         237
  C:00D1H         LINE#         238
  C:00D1H         LINE#         239
  C:00D3H         LINE#         240
  C:00D3H         LINE#         241
  C:00E6H         LINE#         242
  C:0101H         LINE#         243
  C:0101H         LINE#         244
  C:0104H         LINE#         245
  C:0104H         LINE#         246
  C:0104H         LINE#         247
  C:0107H         LINE#         248
  C:0107H         LINE#         249
  C:010AH         LINE#         250
  C:010AH         LINE#         251
  C:010DH         LINE#         257
  C:010DH         LINE#         258
  C:0110H         LINE#         259
  C:0110H         LINE#         260
  C:0113H         LINE#         261
  C:0113H         LINE#         262
  C:0116H         LINE#         263
  C:0116H         LINE#         264
  C:0119H         LINE#         265
  C:0119H         LINE#         266
  C:012CH         LINE#         267
  C:0140H         LINE#         268
  C:0140H         LINE#         269
  C:0140H         LINE#         270
  C:0140H         LINE#         271
  C:0143H         LINE#         272
  C:0143H         LINE#         273
  C:0156H         LINE#         274
  C:0159H         LINE#         275
  C:015CH         LINE#         276
  C:015CH         LINE#         277
  C:015EH         LINE#         283
  C:015EH         LINE#         284
  C:016FH         LINE#         285
  C:016FH         LINE#         286
  C:016FH         LINE#         287
  C:0172H         LINE#         289
  C:0172H         LINE#         290
  C:0172H         LINE#         291
  C:0172H         LINE#         292
  C:0175H         LINE#         293
  C:0175H         LINE#         294
  C:0188H         LINE#         295
  C:0199H         LINE#         296
BL51 BANKED LINKER/LOCATER V6.22                                                      05/19/2022  10:01:03  PAGE 10


  C:0199H         LINE#         297
  C:0199H         LINE#         298
  C:019CH         LINE#         300
  C:019CH         LINE#         301
  C:019CH         LINE#         302
  C:019CH         LINE#         303
  C:019FH         LINE#         304
  C:019FH         LINE#         305
  C:01B2H         LINE#         306
  C:01B5H         LINE#         307
  C:01B8H         LINE#         308
  C:01BBH         LINE#         309
  C:01BEH         LINE#         310
  C:01BEH         LINE#         311
  C:01C1H         LINE#         312
  C:01C4H         LINE#         313
  C:01C7H         LINE#         314
  C:01CAH         LINE#         320
  C:01CAH         LINE#         321
  C:01DDH         LINE#         322
  C:01EEH         LINE#         323
  C:01EEH         LINE#         324
  C:01EEH         LINE#         325
  C:01F0H         LINE#         327
  C:01F0H         LINE#         328
  C:01F0H         LINE#         329
  C:01F0H         LINE#         330
  C:01F2H         LINE#         331
  C:01F2H         LINE#         332
  C:0205H         LINE#         333
  C:0216H         LINE#         334
  C:0216H         LINE#         335
  C:0216H         LINE#         336
  C:0218H         LINE#         338
  C:0218H         LINE#         339
  C:0218H         LINE#         340
  C:0218H         LINE#         341
  C:021AH         LINE#         342
  C:021AH         LINE#         343
  C:022DH         LINE#         344
  C:023EH         LINE#         345
  C:023EH         LINE#         346
  C:0241H         LINE#         347
  C:0243H         LINE#         349
  C:0243H         LINE#         350
  C:0246H         LINE#         351
  C:0246H         LINE#         352
  C:0248H         LINE#         353
  C:0248H         LINE#         354
  C:024BH         LINE#         355
  C:024EH         LINE#         356
  C:0250H         LINE#         357
  C:0250H         LINE#         358
  C:0253H         LINE#         359
  C:0256H         LINE#         360
  C:0258H         LINE#         362
  C:0258H         LINE#         363
BL51 BANKED LINKER/LOCATER V6.22                                                      05/19/2022  10:01:03  PAGE 11


  C:025BH         LINE#         364
  C:025EH         LINE#         365
  C:025EH         LINE#         366
  C:025EH         LINE#         369
  C:0261H         LINE#         370
  -------         ENDPROC       I2C_EXECUTETRANSMISSION
  -------         PROC          ISR_I2C
  C:03D5H         LINE#         376
  C:03EAH         LINE#         378
  C:03EDH         LINE#         379
  -------         ENDPROC       ISR_I2C
  -------         ENDMOD        I2C

  -------         MODULE        OPTIONS_SN8F5835
  C:7FF0H         PUBLIC        CRC_CHECK_DATA
  N:001EH         SYMBOL        BIT16_BYPASS1P_H
  N:00AFH         SYMBOL        BIT16_BYPASS1P_L
  N:0008H         SYMBOL        CK_FINE_TUNING_SET
  N:0018H         SYMBOL        CLOCKSRC_SET
  N:00C0H         SYMBOL        EXTERNAL_CLOCKRATE_SET
  N:00A0H         SYMBOL        IHRC32M_CLOCKRATE_SET
  N:0004H         SYMBOL        ISP_EN_SET
  N:0001H         SYMBOL        NOISEFILT_SET
  N:0030H         SYMBOL        RESETPIN_SET
  N:8000H         SYMBOL        ROM_SIZE
  N:0003H         SYMBOL        SECURITY_SET
  N:00C0H         SYMBOL        WATCHCLK_SET
  N:00A0H         SYMBOL        WATCHDOG_SET
  N:00C0H         SYMBOL        XTAL12M_CLOCKRATE_SET
  N:00E0H         SYMBOL        XTAL4M_CLOCKRATE_SET
  -------         ENDMOD        OPTIONS_SN8F5835

  -------         MODULE        ?C?CLDPTR
  C:034DH         PUBLIC        ?C?CLDPTR
  -------         ENDMOD        ?C?CLDPTR

  -------         MODULE        ?C?CSTPTR
  C:0366H         PUBLIC        ?C?CSTPTR
  -------         ENDMOD        ?C?CSTPTR

  -------         MODULE        ?C?CCASE
  C:0378H         PUBLIC        ?C?CCASE
  -------         ENDMOD        ?C?CCASE

Program Size: data=66.1 xdata=50 code=1202
LINK/LOCATE RUN COMPLETE.  0 WARNING(S),  0 ERROR(S)
